 setnotif001

 Timestamp is c55e9395 (reproducible build file hash)

 Preferred load address is 0000000180000000

 Start         Length     Name                   Class
 0001:00000000 000036a0H .text$mn                CODE
 0001:000036a0 00000036H .text$mn$00             CODE
 0001:000036d6 00000092H .text$x                 CODE
 0002:00000000 00000198H .idata$5                DATA
 0002:00000198 00000038H .00cfg                  DATA
 0002:000001d0 00000008H .CRT$XCA                DATA
 0002:000001d8 00000008H .CRT$XCZ                DATA
 0002:000001e0 00000008H .CRT$XIA                DATA
 0002:000001e8 00000008H .CRT$XIC                DATA
 0002:000001f0 00000008H .CRT$XIZ                DATA
 0002:000001f8 00000008H .CRT$XLA                DATA
 0002:00000200 00000008H .CRT$XLZ                DATA
 0002:00000208 00000008H .CRT$XPA                DATA
 0002:00000210 00000008H .CRT$XPZ                DATA
 0002:00000218 00000008H .CRT$XTA                DATA
 0002:00000220 00000010H .CRT$XTZ                DATA
 0002:00000228 00000000H .gehcont$y              DATA
 0002:00000228 00000000H .gfids$y                DATA
 0002:00000230 00002150H .rdata                  DATA
 0002:00002380 00000000H .rdata$CastGuardVftablesA DATA
 0002:00002380 00000000H .rdata$CastGuardVftablesC DATA
 0002:00002380 00000028H .rdata$T                DATA
 0002:000023a8 000000a4H .rdata$voltmd           DATA
 0002:0000244c 0000031cH .rdata$zzzdbg           DATA
 0002:00002768 00000008H .rtc$IAA                DATA
 0002:00002770 00000008H .rtc$IZZ                DATA
 0002:00002778 00000008H .rtc$TAA                DATA
 0002:00002780 00000008H .rtc$TZZ                DATA
 0002:00002788 00000004H .tls                    DATA
 0002:0000278c 00000004H .tls$                   DATA
 0002:00002790 00000008H .tls$ZZZ                DATA
 0002:00002798 00000318H .xdata                  DATA
 0002:00002ab0 000003f0H .edata                  DATA
 0002:00002ea0 00000064H .idata$2                DATA
 0002:00002f04 00000014H .idata$3                DATA
 0002:00002f18 00000198H .idata$4                DATA
 0002:000030b0 0000041eH .idata$6                DATA
 0003:00000000 00000080H .data                   DATA
 0003:00000080 0001b458H .bss                    DATA
 0004:00000000 0000045cH .pdata                  DATA

  Address         Publics by Value              Rva+Base               Lib:Object

 0000:00000000       __AbsoluteZero             0000000000000000     <absolute>
 0000:00000000       ___safe_se_handler_count   0000000000000000     <absolute>
 0000:00000000       ___safe_se_handler_table   0000000000000000     <absolute>
 0000:00000000       __arm64x_extra_rfe_table   0000000000000000     <absolute>
 0000:00000000       __arm64x_extra_rfe_table_size 0000000000000000     <absolute>
 0000:00000000       __arm64x_native_entrypoint 0000000000000000     <absolute>
 0000:00000000       __arm64x_redirection_metadata 0000000000000000     <absolute>
 0000:00000000       __arm64x_redirection_metadata_count 0000000000000000     <absolute>
 0000:00000000       __dynamic_value_reloc_table 0000000000000000     <absolute>
 0000:00000000       __enclave_config           0000000000000000     <absolute>
 0000:00000000       __guard_check_icall_a64n_fptr 0000000000000000     <absolute>
 0000:00000000       __guard_eh_cont_count      0000000000000000     <absolute>
 0000:00000000       __guard_eh_cont_table      0000000000000000     <absolute>
 0000:00000000       __guard_fids_count         0000000000000000     <absolute>
 0000:00000000       __guard_fids_table         0000000000000000     <absolute>
 0000:00000000       __guard_iat_count          0000000000000000     <absolute>
 0000:00000000       __guard_iat_table          0000000000000000     <absolute>
 0000:00000000       __guard_longjmp_count      0000000000000000     <absolute>
 0000:00000000       __guard_longjmp_table      0000000000000000     <absolute>
 0000:00000000       __hybrid_auxiliary_iat     0000000000000000     <absolute>
 0000:00000000       __hybrid_auxiliary_iat_copy 0000000000000000     <absolute>
 0000:00000000       __hybrid_code_map          0000000000000000     <absolute>
 0000:00000000       __hybrid_code_map_count    0000000000000000     <absolute>
 0000:00000000       __x64_code_ranges_to_entry_points 0000000000000000     <absolute>
 0000:00000000       __x64_code_ranges_to_entry_points_count 0000000000000000     <absolute>
 0000:00000100       __guard_flags              0000000000000100     <absolute>
 0000:00000000       __ImageBase                0000000180000000     <linker-defined>
 0001:00000000       ?NewObject@JNIEnv_@@QEAAPEAV_jobject@@PEAV_jclass@@PEAU_jmethodID@@ZZ 0000000180001000 f i libsetnotif001.obj
 0001:00000028       ?SetEventNotificationMode@_jvmtiEnv@@QEAA?AW4jvmtiError@@W4jvmtiEventMode@@W4jvmtiEvent@@PEAV_jobject@@ZZ 0000000180001028 f i libsetnotif001.obj
 0001:00000034       ?TranslateError@@YAPEBDW4jvmtiError@@@Z 0000000180001034 f   libsetnotif001.obj
 0001:000002ec       ?TranslateEvent@@YAPEBDW4jvmtiEvent@@@Z 00000001800012ec f   libsetnotif001.obj
 0001:00000490       ?nsk_jni_check_exception@@YAHPEAUJNIEnv_@@QEBDH@Z 0000000180001490 f   libsetnotif001.obj
 0001:000005d4       ?nsk_jni_lverify@@YAHHPEAUJNIEnv_@@HQEBDH1ZZ 00000001800015d4 f   libsetnotif001.obj
 0001:00000674       Agent_Initialize           0000000180001674 f   libsetnotif001.obj
 0001:00000980       Agent_OnAttach             0000000180001980 f   libsetnotif001.obj
 0001:00000980       Agent_OnLoad               0000000180001980 f   libsetnotif001.obj
 0001:00000988       Breakpoint                 0000000180001988 f   libsetnotif001.obj
 0001:000009a4       ClassLoad                  00000001800019a4 f   libsetnotif001.obj
 0001:000009c0       ClassPrepare               00000001800019c0 f   libsetnotif001.obj
 0001:000009dc       Exception                  00000001800019dc f   libsetnotif001.obj
 0001:000009f8       ExceptionCatch             00000001800019f8 f   libsetnotif001.obj
 0001:00000a14       FieldAccess                0000000180001a14 f   libsetnotif001.obj
 0001:00000a30       FieldModification          0000000180001a30 f   libsetnotif001.obj
 0001:00000a4c       FramePop                   0000000180001a4c f   libsetnotif001.obj
 0001:00000a68       Java_nsk_jvmti_SetEventNotificationMode_setnotif001_enableEv 0000000180001a68 f   libsetnotif001.obj
 0001:00000af4       Java_nsk_jvmti_SetEventNotificationMode_setnotif001_getRes 0000000180001af4 f   libsetnotif001.obj
 0001:00000ba4       Java_nsk_jvmti_unit_FollowReferences_FollowRefObjects_addRefToVerify 0000000180001ba4 f   libsetnotif001.obj
 0001:00000d7c       Java_nsk_jvmti_unit_FollowReferences_FollowRefObjects_getTag 0000000180001d7c f   libsetnotif001.obj
 0001:00000e3c       Java_nsk_jvmti_unit_FollowReferences_FollowRefObjects_resetRefsToVerify 0000000180001e3c f   libsetnotif001.obj
 0001:00000e44       Java_nsk_jvmti_unit_FollowReferences_FollowRefObjects_resetTags 0000000180001e44 f   libsetnotif001.obj
 0001:00000e88       Java_nsk_jvmti_unit_FollowReferences_FollowRefObjects_setTag 0000000180001e88 f   libsetnotif001.obj
 0001:000010e0       Java_nsk_share_jvmti_ArgumentHandler_getAgentOptionsString 00000001800020e0 f   libsetnotif001.obj
 0001:00001190       Java_nsk_share_jvmti_DebugeeClass_checkStatus 0000000180002190 f   libsetnotif001.obj
 0001:00001218       Java_nsk_share_jvmti_DebugeeClass_resetAgentData 0000000180002218 f   libsetnotif001.obj
 0001:00001278       Java_nsk_share_jvmti_RedefineAgent_agentStatus 0000000180002278 f   libsetnotif001.obj
 0001:00001284       Java_nsk_share_jvmti_RedefineAgent_isRedefined 0000000180002284 f   libsetnotif001.obj
 0001:00001290       Java_nsk_share_jvmti_RedefineAgent_redefineAttempted 0000000180002290 f   libsetnotif001.obj
 0001:0000129c       MA_checkStatus             000000018000229c f   libsetnotif001.obj
 0001:00001340       MethodEntry                0000000180002340 f   libsetnotif001.obj
 0001:00001468       MethodExit                 0000000180002468 f   libsetnotif001.obj
 0001:00001498       SingleStep                 0000000180002498 f   libsetnotif001.obj
 0001:000014c8       ThreadEnd                  00000001800024c8 f   libsetnotif001.obj
 0001:000014e4       ThreadStart                00000001800024e4 f   libsetnotif001.obj
 0001:00001500       VMInit                     0000000180002500 f   libsetnotif001.obj
 0001:00001564       __local_stdio_printf_options 0000000180002564 f i libsetnotif001.obj
 0001:00001744       disable                    0000000180002744 f   libsetnotif001.obj
 0001:000017d0       enable                     00000001800027d0 f   libsetnotif001.obj
 0001:000018f4       exitOnError                00000001800028f4 f   libsetnotif001.obj
 0001:000019a8       fprintf                    00000001800029a8 f i libsetnotif001.obj
 0001:000019ec       mark                       00000001800029ec f   libsetnotif001.obj
 0001:00001afc       nsk_jvmti_lverify          0000000180002afc f   libsetnotif001.obj
 0001:00001bec       nsk_jvmti_resetAgentData   0000000180002bec f   libsetnotif001.obj
 0001:00001c6c       nsk_jvmti_setFailStatus    0000000180002c6c f   libsetnotif001.obj
 0001:00001ca8       nsk_lcomplain              0000000180002ca8 f   libsetnotif001.obj
 0001:00001cc8       nsk_ldisplay               0000000180002cc8 f   libsetnotif001.obj
 0001:00001ce8       nsk_ltrace                 0000000180002ce8 f   libsetnotif001.obj
 0001:00001d08       nsk_lvcomplain             0000000180002d08 f   libsetnotif001.obj
 0001:00001ec0       nsk_lvdisplay              0000000180002ec0 f   libsetnotif001.obj
 0001:00001f0c       nsk_lverify                0000000180002f0c f   libsetnotif001.obj
 0001:00001f68       nsk_lvtrace                0000000180002f68 f   libsetnotif001.obj
 0001:00001fc8       nsk_printf                 0000000180002fc8 f   libsetnotif001.obj
 0001:00001ff0       nsk_vprintf                0000000180002ff0 f   libsetnotif001.obj
 0001:000020a4       printf                     00000001800030a4 f i libsetnotif001.obj
 0001:000020f4       setWatches                 00000001800030f4 f   libsetnotif001.obj
 0001:00002780       __raise_securityfailure    0000000180003780 f   MSVCRT:gs_report.obj
 0001:000027b4       __report_gsfailure         00000001800037b4 f   MSVCRT:gs_report.obj
 0001:000029f4       __GSHandlerCheck           00000001800039f4 f   MSVCRT:gshandler.obj
 0001:00002a14       __GSHandlerCheckCommon     0000000180003a14 f   MSVCRT:gshandler.obj
 0001:00002a80       __security_check_cookie    0000000180003a80 f   MSVCRT:amdsecgs.obj
 0001:00002dc0       _DllMainCRTStartup         0000000180003dc0 f   MSVCRT:dll_dllmain.obj
 0001:00002e00       __scrt_acquire_startup_lock 0000000180003e00 f   MSVCRT:utility.obj
 0001:00002e3c       __scrt_dllmain_after_initialize_c 0000000180003e3c f   MSVCRT:utility.obj
 0001:00002e70       __scrt_dllmain_before_initialize_c 0000000180003e70 f   MSVCRT:utility.obj
 0001:00002e88       __scrt_dllmain_crt_thread_attach 0000000180003e88 f   MSVCRT:utility.obj
 0001:00002eb0       __scrt_dllmain_crt_thread_detach 0000000180003eb0 f   MSVCRT:utility.obj
 0001:00002ec8       __scrt_dllmain_exception_filter 0000000180003ec8 f   MSVCRT:utility.obj
 0001:00002f28       __scrt_dllmain_uninitialize_c 0000000180003f28 f   MSVCRT:utility.obj
 0001:00002f58       __scrt_dllmain_uninitialize_critical 0000000180003f58 f   MSVCRT:utility.obj
 0001:00002f6c       __scrt_initialize_crt      0000000180003f6c f   MSVCRT:utility.obj
 0001:00002fb8       __scrt_initialize_onexit_tables 0000000180003fb8 f   MSVCRT:utility.obj
 0001:00003044       __scrt_is_nonwritable_in_current_image 0000000180004044 f   MSVCRT:utility.obj
 0001:000030dc       __scrt_release_startup_lock 00000001800040dc f   MSVCRT:utility.obj
 0001:00003100       __scrt_uninitialize_crt    0000000180004100 f   MSVCRT:utility.obj
 0001:0000312c       _onexit                    000000018000412c f   MSVCRT:utility.obj
 0001:00003168       atexit                     0000000180004168 f   MSVCRT:utility.obj
 0001:00003180       __crt_debugger_hook        0000000180004180 f   MSVCRT:utility_desktop.obj
 0001:00003188       __scrt_fastfail            0000000180004188 f   MSVCRT:utility_desktop.obj
 0001:000032d4       _guard_check_icall_nop     00000001800042d4 f i MSVCRT:guard_support.obj
 0001:000032d8       __security_init_cookie     00000001800042d8 f   MSVCRT:gs_support.obj
 0001:00003384       DllMain                    0000000180004384 f   MSVCRT:dll_dllmain_stub.obj
 0001:000033a8       ?__scrt_initialize_type_info@@YAXXZ 00000001800043a8 f   MSVCRT:tncleanup.obj
 0001:000033b8       ?__scrt_uninitialize_type_info@@YAXXZ 00000001800043b8 f   MSVCRT:tncleanup.obj
 0001:000033c4       __local_stdio_scanf_options 00000001800043c4 f i MSVCRT:default_local_stdio_options.obj
 0001:000033cc       __scrt_initialize_default_local_stdio_options 00000001800043cc f   MSVCRT:default_local_stdio_options.obj
 0001:000033e8       __scrt_get_dyn_tls_init_callback 00000001800043e8 f   MSVCRT:dyn_tls_init.obj
 0001:000033f0       _RTC_Initialize            00000001800043f0 f   MSVCRT:initsect.obj
 0001:0000342c       _RTC_Terminate             000000018000442c f   MSVCRT:initsect.obj
 0001:00003468       __isa_available_init       0000000180004468 f   MSVCRT:cpu_disp.obj
 0001:00003614       _get_startup_argv_mode     0000000180004614 f   MSVCRT:argv_mode.obj
 0001:0000361c       __scrt_is_ucrt_dll_in_use  000000018000461c f   MSVCRT:ucrt_detection.obj
 0001:00003630       memcpy                     0000000180004630 f   vcruntime:VCRUNTIME140.dll
 0001:00003636       memset                     0000000180004636 f   vcruntime:VCRUNTIME140.dll
 0001:0000363c       strchr                     000000018000463c f   vcruntime:VCRUNTIME140.dll
 0001:00003642       __C_specific_handler       0000000180004642 f   vcruntime:VCRUNTIME140.dll
 0001:00003648       __std_type_info_destroy_list 0000000180004648 f   vcruntime:VCRUNTIME140.dll
 0001:0000364e       strcmp                     000000018000464e f   ucrt:api-ms-win-crt-string-l1-1-0.dll
 0001:00003654       strlen                     0000000180004654 f   ucrt:api-ms-win-crt-string-l1-1-0.dll
 0001:0000365a       _initterm                  000000018000465a f   ucrt:api-ms-win-crt-runtime-l1-1-0.dll
 0001:00003660       _initterm_e                0000000180004660 f   ucrt:api-ms-win-crt-runtime-l1-1-0.dll
 0001:00003666       _seh_filter_dll            0000000180004666 f   ucrt:api-ms-win-crt-runtime-l1-1-0.dll
 0001:0000366c       _configure_narrow_argv     000000018000466c f   ucrt:api-ms-win-crt-runtime-l1-1-0.dll
 0001:00003672       _initialize_narrow_environment 0000000180004672 f   ucrt:api-ms-win-crt-runtime-l1-1-0.dll
 0001:00003678       _initialize_onexit_table   0000000180004678 f   ucrt:api-ms-win-crt-runtime-l1-1-0.dll
 0001:0000367e       _register_onexit_function  000000018000467e f   ucrt:api-ms-win-crt-runtime-l1-1-0.dll
 0001:00003684       _execute_onexit_table      0000000180004684 f   ucrt:api-ms-win-crt-runtime-l1-1-0.dll
 0001:0000368a       _crt_atexit                000000018000468a f   ucrt:api-ms-win-crt-runtime-l1-1-0.dll
 0001:00003690       _cexit                     0000000180004690 f   ucrt:api-ms-win-crt-runtime-l1-1-0.dll
 0001:00003698       __acrt_initialize          0000000180004698 f   MSVCRT:ucrt_stubs.obj
 0001:00003698       __acrt_thread_attach       0000000180004698 f   MSVCRT:ucrt_stubs.obj
 0001:00003698       __acrt_thread_detach       0000000180004698 f   MSVCRT:ucrt_stubs.obj
 0001:00003698       __acrt_uninitialize        0000000180004698 f   MSVCRT:ucrt_stubs.obj
 0001:00003698       __acrt_uninitialize_critical 0000000180004698 f   MSVCRT:ucrt_stubs.obj
 0001:00003698       __scrt_stub_for_acrt_initialize 0000000180004698 f   MSVCRT:ucrt_stubs.obj
 0001:00003698       __scrt_stub_for_acrt_thread_attach 0000000180004698 f   MSVCRT:ucrt_stubs.obj
 0001:00003698       __scrt_stub_for_acrt_thread_detach 0000000180004698 f   MSVCRT:ucrt_stubs.obj
 0001:00003698       __scrt_stub_for_acrt_uninitialize 0000000180004698 f   MSVCRT:ucrt_stubs.obj
 0001:00003698       __scrt_stub_for_acrt_uninitialize_critical 0000000180004698 f   MSVCRT:ucrt_stubs.obj
 0001:00003698       __vcrt_initialize          0000000180004698 f   MSVCRT:ucrt_stubs.obj
 0001:00003698       __vcrt_thread_attach       0000000180004698 f   MSVCRT:ucrt_stubs.obj
 0001:00003698       __vcrt_thread_detach       0000000180004698 f   MSVCRT:ucrt_stubs.obj
 0001:00003698       __vcrt_uninitialize        0000000180004698 f   MSVCRT:ucrt_stubs.obj
 0001:00003698       __vcrt_uninitialize_critical 0000000180004698 f   MSVCRT:ucrt_stubs.obj
 0001:0000369c       __scrt_stub_for_is_c_termination_complete 000000018000469c f   MSVCRT:ucrt_stubs.obj
 0001:0000369c       _is_c_termination_complete 000000018000469c f   MSVCRT:ucrt_stubs.obj
 0001:000036b0       _guard_dispatch_icall_nop  00000001800046b0 f   MSVCRT:guard_dispatch.obj
 0001:000036d0       _guard_xfg_dispatch_icall_nop 00000001800046d0 f   MSVCRT:guard_xfg_dispatch.obj
 0002:00000000       __imp_RtlCaptureContext    0000000180005000     kernel32:KERNEL32.dll
 0002:00000008       __imp_RtlLookupFunctionEntry 0000000180005008     kernel32:KERNEL32.dll
 0002:00000010       __imp_RtlVirtualUnwind     0000000180005010     kernel32:KERNEL32.dll
 0002:00000018       __imp_UnhandledExceptionFilter 0000000180005018     kernel32:KERNEL32.dll
 0002:00000020       __imp_SetUnhandledExceptionFilter 0000000180005020     kernel32:KERNEL32.dll
 0002:00000028       __imp_GetCurrentProcess    0000000180005028     kernel32:KERNEL32.dll
 0002:00000030       __imp_TerminateProcess     0000000180005030     kernel32:KERNEL32.dll
 0002:00000038       __imp_IsProcessorFeaturePresent 0000000180005038     kernel32:KERNEL32.dll
 0002:00000040       __imp_CloseHandle          0000000180005040     kernel32:KERNEL32.dll
 0002:00000048       __imp_InitializeCriticalSectionAndSpinCount 0000000180005048     kernel32:KERNEL32.dll
 0002:00000050       __imp_DeleteCriticalSection 0000000180005050     kernel32:KERNEL32.dll
 0002:00000058       __imp_CreateEventW         0000000180005058     kernel32:KERNEL32.dll
 0002:00000060       __imp_GetModuleHandleW     0000000180005060     kernel32:KERNEL32.dll
 0002:00000068       __imp_GetProcAddress       0000000180005068     kernel32:KERNEL32.dll
 0002:00000070       __imp_IsDebuggerPresent    0000000180005070     kernel32:KERNEL32.dll
 0002:00000078       __imp_QueryPerformanceCounter 0000000180005078     kernel32:KERNEL32.dll
 0002:00000080       __imp_GetCurrentProcessId  0000000180005080     kernel32:KERNEL32.dll
 0002:00000088       __imp_GetCurrentThreadId   0000000180005088     kernel32:KERNEL32.dll
 0002:00000090       __imp_GetSystemTimeAsFileTime 0000000180005090     kernel32:KERNEL32.dll
 0002:00000098       __imp_DisableThreadLibraryCalls 0000000180005098     kernel32:KERNEL32.dll
 0002:000000a0       __imp_InitializeSListHead  00000001800050a0     kernel32:KERNEL32.dll
 0002:000000a8       \177KERNEL32_NULL_THUNK_DATA 00000001800050a8     kernel32:KERNEL32.dll
 0002:000000b0       __imp_memcpy               00000001800050b0     vcruntime:VCRUNTIME140.dll
 0002:000000b8       __imp_memset               00000001800050b8     vcruntime:VCRUNTIME140.dll
 0002:000000c0       __imp_strchr               00000001800050c0     vcruntime:VCRUNTIME140.dll
 0002:000000c8       __imp___C_specific_handler 00000001800050c8     vcruntime:VCRUNTIME140.dll
 0002:000000d0       __imp___std_type_info_destroy_list 00000001800050d0     vcruntime:VCRUNTIME140.dll
 0002:000000d8       \177VCRUNTIME140_NULL_THUNK_DATA 00000001800050d8     vcruntime:VCRUNTIME140.dll
 0002:000000e0       __imp__errno               00000001800050e0     ucrt:api-ms-win-crt-runtime-l1-1-0.dll
 0002:000000e8       __imp_exit                 00000001800050e8     ucrt:api-ms-win-crt-runtime-l1-1-0.dll
 0002:000000f0       __imp__cexit               00000001800050f0     ucrt:api-ms-win-crt-runtime-l1-1-0.dll
 0002:000000f8       __imp__crt_atexit          00000001800050f8     ucrt:api-ms-win-crt-runtime-l1-1-0.dll
 0002:00000100       __imp__execute_onexit_table 0000000180005100     ucrt:api-ms-win-crt-runtime-l1-1-0.dll
 0002:00000108       __imp__register_onexit_function 0000000180005108     ucrt:api-ms-win-crt-runtime-l1-1-0.dll
 0002:00000110       __imp__initialize_onexit_table 0000000180005110     ucrt:api-ms-win-crt-runtime-l1-1-0.dll
 0002:00000118       __imp__initialize_narrow_environment 0000000180005118     ucrt:api-ms-win-crt-runtime-l1-1-0.dll
 0002:00000120       __imp__configure_narrow_argv 0000000180005120     ucrt:api-ms-win-crt-runtime-l1-1-0.dll
 0002:00000128       __imp__seh_filter_dll      0000000180005128     ucrt:api-ms-win-crt-runtime-l1-1-0.dll
 0002:00000130       __imp__initterm_e          0000000180005130     ucrt:api-ms-win-crt-runtime-l1-1-0.dll
 0002:00000138       __imp__initterm            0000000180005138     ucrt:api-ms-win-crt-runtime-l1-1-0.dll
 0002:00000140       \177api-ms-win-crt-runtime-l1-1-0_NULL_THUNK_DATA 0000000180005140     ucrt:api-ms-win-crt-runtime-l1-1-0.dll
 0002:00000148       __imp___acrt_iob_func      0000000180005148     ucrt:api-ms-win-crt-stdio-l1-1-0.dll
 0002:00000150       __imp_fflush               0000000180005150     ucrt:api-ms-win-crt-stdio-l1-1-0.dll
 0002:00000158       __imp___stdio_common_vsprintf 0000000180005158     ucrt:api-ms-win-crt-stdio-l1-1-0.dll
 0002:00000160       __imp___stdio_common_vfprintf 0000000180005160     ucrt:api-ms-win-crt-stdio-l1-1-0.dll
 0002:00000168       \177api-ms-win-crt-stdio-l1-1-0_NULL_THUNK_DATA 0000000180005168     ucrt:api-ms-win-crt-stdio-l1-1-0.dll
 0002:00000170       __imp_strcmp               0000000180005170     ucrt:api-ms-win-crt-string-l1-1-0.dll
 0002:00000178       __imp__strdup              0000000180005178     ucrt:api-ms-win-crt-string-l1-1-0.dll
 0002:00000178       __imp_strdup               0000000180005178     ucrt:api-ms-win-crt-string-l1-1-0.dll
 0002:00000180       __imp_strlen               0000000180005180     ucrt:api-ms-win-crt-string-l1-1-0.dll
 0002:00000188       __imp_strncpy              0000000180005188     ucrt:api-ms-win-crt-string-l1-1-0.dll
 0002:00000190       \177api-ms-win-crt-string-l1-1-0_NULL_THUNK_DATA 0000000180005190     ucrt:api-ms-win-crt-string-l1-1-0.dll
 0002:00000198       __guard_check_icall_fptr   0000000180005198     MSVCRT:guard_support.obj
 0002:000001a0       __guard_xfg_check_icall_fptr 00000001800051a0     MSVCRT:guard_support.obj
 0002:000001a8       __guard_dispatch_icall_fptr 00000001800051a8     MSVCRT:guard_support.obj
 0002:000001b0       __guard_xfg_dispatch_icall_fptr 00000001800051b0     MSVCRT:guard_support.obj
 0002:000001b8       __guard_xfg_table_dispatch_icall_fptr 00000001800051b8     MSVCRT:guard_support.obj
 0002:000001c0       __castguard_check_failure_os_handled_fptr 00000001800051c0     MSVCRT:guard_support.obj
 0002:000001c8       __guard_memcpy_fptr        00000001800051c8     vcruntime:softmemtag.obj
 0002:000001d0       __xc_a                     00000001800051d0     MSVCRT:initializers.obj
 0002:000001d8       __xc_z                     00000001800051d8     MSVCRT:initializers.obj
 0002:000001e0       __xi_a                     00000001800051e0     MSVCRT:initializers.obj
 0002:000001f0       __xi_z                     00000001800051f0     MSVCRT:initializers.obj
 0002:000001f8       __xl_a                     00000001800051f8     MSVCRT:tlssup.obj
 0002:00000200       __xl_z                     0000000180005200     MSVCRT:tlssup.obj
 0002:00000208       __xp_a                     0000000180005208     MSVCRT:initializers.obj
 0002:00000210       __xp_z                     0000000180005210     MSVCRT:initializers.obj
 0002:00000218       __xt_a                     0000000180005218     MSVCRT:initializers.obj
 0002:00000220       __xt_z                     0000000180005220     MSVCRT:initializers.obj
 0002:00000230       g_refKindStr               0000000180005230     libsetnotif001.obj
 0002:000003e0       ??_C@_09BPLDFGCI@unknown_0@ 00000001800053e0     libsetnotif001.obj
 0002:000003f0       ??_C@_0BL@FPNMECJD@JVMTI_HEAP_REFERENCE_CLASS@ 00000001800053f0     libsetnotif001.obj
 0002:00000410       ??_C@_0BL@FKGKKLNM@JVMTI_HEAP_REFERENCE_FIELD@ 0000000180005410     libsetnotif001.obj
 0002:00000430       ??_C@_0CD@CAEHCFJF@JVMTI_HEAP_REFERENCE_ARRAY_ELEM@ 0000000180005430     libsetnotif001.obj
 0002:00000458       ??_C@_0CC@DNEBMCNK@JVMTI_HEAP_REFERENCE_CLASS_LOAD@ 0000000180005458     libsetnotif001.obj
 0002:00000480       ??_C@_0BN@CJMIPEBB@JVMTI_HEAP_REFERENCE_SIGNERS@ 0000000180005480     libsetnotif001.obj
 0002:000004a0       ??_C@_0CH@HBOIDPEB@JVMTI_HEAP_REFERENCE_PROTECTION@ 00000001800054a0     libsetnotif001.obj
 0002:000004c8       ??_C@_0BP@MDKGDGKL@JVMTI_HEAP_REFERENCE_INTERFACE@ 00000001800054c8     libsetnotif001.obj
 0002:000004e8       ??_C@_0CC@JJMIHNJH@JVMTI_HEAP_REFERENCE_STATIC_FIE@ 00000001800054e8     libsetnotif001.obj
 0002:00000510       ??_C@_0CD@IDHEEGID@JVMTI_HEAP_REFERENCE_CONSTANT_P@ 0000000180005510     libsetnotif001.obj
 0002:00000538       ??_C@_0CA@EFFCHNG@JVMTI_HEAP_REFERENCE_SUPERCLASS@ 0000000180005538     libsetnotif001.obj
 0002:00000558       ??_C@_0L@PCDFHGCJ@unknown_11@ 0000000180005558     libsetnotif001.obj
 0002:00000568       ??_C@_0L@NJBICFOK@unknown_12@ 0000000180005568     libsetnotif001.obj
 0002:00000578       ??_C@_0L@MAADBEKL@unknown_13@ 0000000180005578     libsetnotif001.obj
 0002:00000588       ??_C@_0L@IPECICGM@unknown_14@ 0000000180005588     libsetnotif001.obj
 0002:00000598       ??_C@_0L@JGFJLDCN@unknown_15@ 0000000180005598     libsetnotif001.obj
 0002:000005a8       ??_C@_0L@LNHEOAOO@unknown_16@ 00000001800055a8     libsetnotif001.obj
 0002:000005b8       ??_C@_0L@KEGPNBKP@unknown_17@ 00000001800055b8     libsetnotif001.obj
 0002:000005c8       ??_C@_0L@CDPHMNGA@unknown_18@ 00000001800055c8     libsetnotif001.obj
 0002:000005d8       ??_C@_0L@DKOMPMCB@unknown_19@ 00000001800055d8     libsetnotif001.obj
 0002:000005e8       ??_C@_0L@OJGIPJDB@unknown_20@ 00000001800055e8     libsetnotif001.obj
 0002:000005f8       ??_C@_0CA@KAOFNDEM@JVMTI_HEAP_REFERENCE_JNI_GLOBAL@ 00000001800055f8     libsetnotif001.obj
 0002:00000618       ??_C@_0CC@HPFAJBK@JVMTI_HEAP_REFERENCE_SYSTEM_CLA@ 0000000180005618     libsetnotif001.obj
 0002:00000640       ??_C@_0BN@FDEGFOHC@JVMTI_HEAP_REFERENCE_MONITOR@ 0000000180005640     libsetnotif001.obj
 0002:00000660       ??_C@_0CB@HKIBCMAJ@JVMTI_HEAP_REFERENCE_STACK_LOCA@ 0000000180005660     libsetnotif001.obj
 0002:00000688       ??_C@_0BP@EAACMMOE@JVMTI_HEAP_REFERENCE_JNI_LOCAL@ 0000000180005688     libsetnotif001.obj
 0002:000006a8       ??_C@_0BM@IJDEOGOE@JVMTI_HEAP_REFERENCE_THREAD@ 00000001800056a8     libsetnotif001.obj
 0002:000006c8       ??_C@_0BL@EDGPPKC@JVMTI_HEAP_REFERENCE_OTHER@ 00000001800056c8     libsetnotif001.obj
 0002:000006e4       ??_C@_04BCJPDBDA@Code@     00000001800056e4     libsetnotif001.obj
 0002:000006f0       ??_C@_0BA@OCLMCFKC@LineNumberTable@ 00000001800056f0     libsetnotif001.obj
 0002:00000700       ??_C@_0BD@CPAEPILC@LocalVariableTable@ 0000000180005700     libsetnotif001.obj
 0002:00000718       ??_C@_0BH@NMBDNHBD@LocalVariableTypeTable@ 0000000180005718     libsetnotif001.obj
 0002:00000730       ??_C@_0O@HIHEEDNJ@StackMapTable@ 0000000180005730     libsetnotif001.obj
 0002:00000740       ??_C@_0L@HCDIAMJG@?9?5?$CFs?0?5?$CFd?3?5@ 0000000180005740     libsetnotif001.obj
 0002:00000750       ??_C@_0JI@HLPECLFI@?$CD?5?4?4?4?6?$CD?5ERROR?3?5too?5many?5complai@ 0000000180005750     libsetnotif001.obj
 0002:000007f0       ??_C@_0ED@JNEKCCOB@The?5following?5fake?5exception?5st@ 00000001800057f0     libsetnotif001.obj
 0002:00000838       ??_C@_0CN@FCNMDFBH@nsk?4share?4Fake_Exception_for_RU@ 0000000180005838     libsetnotif001.obj
 0002:00000868       ??_C@_08PGFFNAEI@?$CI?$CFs?3?$CFd?$CJ?5@ 0000000180005868     libsetnotif001.obj
 0002:00000878       ??_C@_0DP@IENMAEGI@s?2test?2hotspot?2jtreg?2vmTestbase@ 0000000180005878     libsetnotif001.obj
 0002:000008b8       ??_C@_0BL@NDJLFFJB@?7at?5nsk_lvcomplain?$CI?$CFs?3?$CFd?$CJ?6@ 00000001800058b8     libsetnotif001.obj
 0002:000008d8       ??_C@_0BC@JOOKAFKF@?$CD?5ERROR?3?5?$CFs?0?5?$CFd?3?5@ 00000001800058d8     libsetnotif001.obj
 0002:000008f0       ??_C@_09KJEAHMEH@?$CD?5ERROR?3?5@ 00000001800058f0     libsetnotif001.obj
 0002:000008fc       ??_C@_02GPIOPFAK@?$DO?$DO@ 00000001800058fc     libsetnotif001.obj
 0002:00000900       ??_C@_02FODMEDOG@?$DM?$DM@ 0000000180005900     libsetnotif001.obj
 0002:00000904       ??_C@_02DJGKEECL@?4?4@     0000000180005904     libsetnotif001.obj
 0002:00000908       ??_C@_0O@CJPGJOAF@?9?5?$CFs?0?5?$CFd?3?5?$CFs?5@ 0000000180005908     libsetnotif001.obj
 0002:00000918       ??_C@_0CB@IAKPDOIC@?$CD?5?5?5verified?5assertion?5is?5FALSE@ 0000000180005918     libsetnotif001.obj
 0002:00000940       ??_C@_0CO@LGONDEPD@stdout?3?5fflush?5failed?5?9?5err?$DN?$CFd?5@ 0000000180005940     libsetnotif001.obj
 0002:00000970       ??_C@_0CO@KBGKJPBD@stderr?3?5fflush?5failed?5?9?5err?$DN?$CFd?5@ 0000000180005970     libsetnotif001.obj
 0002:000009a0       ??_C@_0BE@JBBKEHHC@JVMTI_EVENT_VM_INIT@ 00000001800059a0     libsetnotif001.obj
 0002:000009b8       ??_C@_0BF@IIMAMFHK@JVMTI_EVENT_VM_DEATH@ 00000001800059b8     libsetnotif001.obj
 0002:000009d0       ??_C@_0BJ@EGBIOBHK@JVMTI_EVENT_THREAD_START@ 00000001800059d0     libsetnotif001.obj
 0002:000009f0       ??_C@_0BH@HCFHMMGI@JVMTI_EVENT_THREAD_END@ 00000001800059f0     libsetnotif001.obj
 0002:00000a08       ??_C@_0CB@NNIAHNJH@JVMTI_EVENT_CLASS_FILE_LOAD_HOO@ 0000000180005a08     libsetnotif001.obj
 0002:00000a30       ??_C@_0BH@JBJMOPG@JVMTI_EVENT_CLASS_LOAD@ 0000000180005a30     libsetnotif001.obj
 0002:00000a48       ??_C@_0BK@GCCJIJJD@JVMTI_EVENT_CLASS_PREPARE@ 0000000180005a48     libsetnotif001.obj
 0002:00000a68       ??_C@_0BF@CJGJGIIE@JVMTI_EVENT_VM_START@ 0000000180005a68     libsetnotif001.obj
 0002:00000a80       ??_C@_0BG@CFCIDKHE@JVMTI_EVENT_EXCEPTION@ 0000000180005a80     libsetnotif001.obj
 0002:00000a98       ??_C@_0BM@BHPDBCCO@JVMTI_EVENT_EXCEPTION_CATCH@ 0000000180005a98     libsetnotif001.obj
 0002:00000ab8       ??_C@_0BI@LDGGDNNG@JVMTI_EVENT_SINGLE_STEP@ 0000000180005ab8     libsetnotif001.obj
 0002:00000ad0       ??_C@_0BG@PHGAMHAA@JVMTI_EVENT_FRAME_POP@ 0000000180005ad0     libsetnotif001.obj
 0002:00000ae8       ??_C@_0BH@BELANHCL@JVMTI_EVENT_BREAKPOINT@ 0000000180005ae8     libsetnotif001.obj
 0002:00000b00       ??_C@_0BJ@DOGOOJAJ@JVMTI_EVENT_FIELD_ACCESS@ 0000000180005b00     libsetnotif001.obj
 0002:00000b20       ??_C@_0BP@NPAIPHIB@JVMTI_EVENT_FIELD_MODIFICATION@ 0000000180005b20     libsetnotif001.obj
 0002:00000b40       ??_C@_0BJ@BDBKGBIC@JVMTI_EVENT_METHOD_ENTRY@ 0000000180005b40     libsetnotif001.obj
 0002:00000b60       ??_C@_0BI@FDJIKCKO@JVMTI_EVENT_METHOD_EXIT@ 0000000180005b60     libsetnotif001.obj
 0002:00000b78       ??_C@_0BP@LONCDEHA@JVMTI_EVENT_NATIVE_METHOD_BIND@ 0000000180005b78     libsetnotif001.obj
 0002:00000b98       ??_C@_0CB@EKPPCCHF@JVMTI_EVENT_COMPILED_METHOD_LOA@ 0000000180005b98     libsetnotif001.obj
 0002:00000bc0       ??_C@_0CD@HEOOKCFG@JVMTI_EVENT_COMPILED_METHOD_UNL@ 0000000180005bc0     libsetnotif001.obj
 0002:00000be8       ??_C@_0CD@MDFNCKBA@JVMTI_EVENT_DYNAMIC_CODE_GENERA@ 0000000180005be8     libsetnotif001.obj
 0002:00000c10       ??_C@_0BO@MDFHOLMG@JVMTI_EVENT_DATA_DUMP_REQUEST@ 0000000180005c10     libsetnotif001.obj
 0002:00000c30       ??_C@_0BJ@EFDJJONH@JVMTI_EVENT_MONITOR_WAIT@ 0000000180005c30     libsetnotif001.obj
 0002:00000c50       ??_C@_0BL@DLIKGNII@JVMTI_EVENT_MONITOR_WAITED@ 0000000180005c50     libsetnotif001.obj
 0002:00000c70       ??_C@_0CE@PFEEOMOD@JVMTI_EVENT_MONITOR_CONTENDED_E@ 0000000180005c70     libsetnotif001.obj
 0002:00000c98       ??_C@_0CG@DOKLDOBC@JVMTI_EVENT_MONITOR_CONTENDED_E@ 0000000180005c98     libsetnotif001.obj
 0002:00000cc0       ??_C@_0CF@KMHIPEGD@JVMTI_EVENT_GARBAGE_COLLECTION_@ 0000000180005cc0     libsetnotif001.obj
 0002:00000ce8       ??_C@_0CG@GGBOHOPN@JVMTI_EVENT_GARBAGE_COLLECTION_@ 0000000180005ce8     libsetnotif001.obj
 0002:00000d10       ??_C@_0BI@BMBPLGPP@JVMTI_EVENT_OBJECT_FREE@ 0000000180005d10     libsetnotif001.obj
 0002:00000d28       ??_C@_0BM@BOCKOKFD@JVMTI_EVENT_VM_OBJECT_ALLOC@ 0000000180005d28     libsetnotif001.obj
 0002:00000d48       ??_C@_0BA@DJDHKMPJ@?$DMunknown?5event?$DO@ 0000000180005d48     libsetnotif001.obj
 0002:00000d58       ??_C@_0BB@JCNMKLLK@JVMTI_ERROR_NONE@ 0000000180005d58     libsetnotif001.obj
 0002:00000d70       ??_C@_0BL@LDIMKLPH@JVMTI_ERROR_INVALID_THREAD@ 0000000180005d70     libsetnotif001.obj
 0002:00000d90       ??_C@_0CB@PJFPAIKJ@JVMTI_ERROR_INVALID_THREAD_GROU@ 0000000180005d90     libsetnotif001.obj
 0002:00000db8       ??_C@_0BN@LLMKHMNF@JVMTI_ERROR_INVALID_PRIORITY@ 0000000180005db8     libsetnotif001.obj
 0002:00000dd8       ??_C@_0CB@MBOFKAGB@JVMTI_ERROR_THREAD_NOT_SUSPENDE@ 0000000180005dd8     libsetnotif001.obj
 0002:00000e00       ??_C@_0BN@FABOLPBI@JVMTI_ERROR_THREAD_SUSPENDED@ 0000000180005e00     libsetnotif001.obj
 0002:00000e20       ??_C@_0BN@FDGNOBJM@JVMTI_ERROR_THREAD_NOT_ALIVE@ 0000000180005e20     libsetnotif001.obj
 0002:00000e40       ??_C@_0BL@GOBIFKNJ@JVMTI_ERROR_INVALID_OBJECT@ 0000000180005e40     libsetnotif001.obj
 0002:00000e60       ??_C@_0BK@FCMAJPPC@JVMTI_ERROR_INVALID_CLASS@ 0000000180005e60     libsetnotif001.obj
 0002:00000e80       ??_C@_0BP@IKLLBKEB@JVMTI_ERROR_CLASS_NOT_PREPARED@ 0000000180005e80     libsetnotif001.obj
 0002:00000ea0       ??_C@_0BN@KLPPLKG@JVMTI_ERROR_INVALID_METHODID@ 0000000180005ea0     libsetnotif001.obj
 0002:00000ec0       ??_C@_0BN@BCEKOKND@JVMTI_ERROR_INVALID_LOCATION@ 0000000180005ec0     libsetnotif001.obj
 0002:00000ee0       ??_C@_0BM@DFDGPME@JVMTI_ERROR_INVALID_FIELDID@ 0000000180005ee0     libsetnotif001.obj
 0002:00000f00       ??_C@_0BL@NELIEPEC@JVMTI_ERROR_NO_MORE_FRAMES@ 0000000180005f00     libsetnotif001.obj
 0002:00000f20       ??_C@_0BJ@BDBECFDM@JVMTI_ERROR_OPAQUE_FRAME@ 0000000180005f20     libsetnotif001.obj
 0002:00000f40       ??_C@_0BK@MIIFNLOB@JVMTI_ERROR_TYPE_MISMATCH@ 0000000180005f40     libsetnotif001.obj
 0002:00000f60       ??_C@_0BJ@HPCAOILC@JVMTI_ERROR_INVALID_SLOT@ 0000000180005f60     libsetnotif001.obj
 0002:00000f80       ??_C@_0BG@CHILOPNI@JVMTI_ERROR_DUPLICATE@ 0000000180005f80     libsetnotif001.obj
 0002:00000f98       ??_C@_0BG@DIEMLHKM@JVMTI_ERROR_NOT_FOUND@ 0000000180005f98     libsetnotif001.obj
 0002:00000fb0       ??_C@_0BM@NHMCKHOB@JVMTI_ERROR_INVALID_MONITOR@ 0000000180005fb0     libsetnotif001.obj
 0002:00000fd0       ??_C@_0BO@PPEDAJGL@JVMTI_ERROR_NOT_MONITOR_OWNER@ 0000000180005fd0     libsetnotif001.obj
 0002:00000ff0       ??_C@_0BG@FCAIPEID@JVMTI_ERROR_INTERRUPT@ 0000000180005ff0     libsetnotif001.obj
 0002:00001008       ??_C@_0CB@EGDBNKOI@JVMTI_ERROR_INVALID_CLASS_FORMA@ 0000000180006008     libsetnotif001.obj
 0002:00001030       ??_C@_0CG@DGKOGIAL@JVMTI_ERROR_CIRCULAR_CLASS_DEFI@ 0000000180006030     libsetnotif001.obj
 0002:00001058       ??_C@_0BP@ICEALPKC@JVMTI_ERROR_FAILS_VERIFICATION@ 0000000180006058     libsetnotif001.obj
 0002:00001078       ??_C@_0DC@JDACLMIO@JVMTI_ERROR_UNSUPPORTED_REDEFIN@ 0000000180006078     libsetnotif001.obj
 0002:000010b0       ??_C@_0DE@GKDKNOMJ@JVMTI_ERROR_UNSUPPORTED_REDEFIN@ 00000001800060b0     libsetnotif001.obj
 0002:000010e8       ??_C@_0BO@LAFKIOG@JVMTI_ERROR_INVALID_TYPESTATE@ 00000001800060e8     libsetnotif001.obj
 0002:00001108       ??_C@_0DH@INDGCLLB@JVMTI_ERROR_UNSUPPORTED_REDEFIN@ 0000000180006108     libsetnotif001.obj
 0002:00001140       ??_C@_0DE@NHEOMMGI@JVMTI_ERROR_UNSUPPORTED_REDEFIN@ 0000000180006140     libsetnotif001.obj
 0002:00001178       ??_C@_0CA@EKPNJOEP@JVMTI_ERROR_UNSUPPORTED_VERSION@ 0000000180006178     libsetnotif001.obj
 0002:00001198       ??_C@_0BN@OFFMAHHL@JVMTI_ERROR_NAMES_DONT_MATCH@ 0000000180006198     libsetnotif001.obj
 0002:000011b8       ??_C@_0DN@HHBBLAKE@JVMTI_ERROR_UNSUPPORTED_REDEFIN@ 00000001800061b8     libsetnotif001.obj
 0002:000011f8       ??_C@_0DO@HMBGBGNA@JVMTI_ERROR_UNSUPPORTED_REDEFIN@ 00000001800061f8     libsetnotif001.obj
 0002:00001238       ??_C@_0BP@PBECGKHJ@JVMTI_ERROR_UNMODIFIABLE_CLASS@ 0000000180006238     libsetnotif001.obj
 0002:00001258       ??_C@_0BK@CANILEHF@JVMTI_ERROR_NOT_AVAILABLE@ 0000000180006258     libsetnotif001.obj
 0002:00001278       ??_C@_0CE@INJKMEFK@JVMTI_ERROR_MUST_POSSESS_CAPABI@ 0000000180006278     libsetnotif001.obj
 0002:000012a0       ??_C@_0BJ@LBFPFPDM@JVMTI_ERROR_NULL_POINTER@ 00000001800062a0     libsetnotif001.obj
 0002:000012c0       ??_C@_0BP@CHJPNNEM@JVMTI_ERROR_ABSENT_INFORMATION@ 00000001800062c0     libsetnotif001.obj
 0002:000012e0       ??_C@_0BP@OMFMNLC@JVMTI_ERROR_INVALID_EVENT_TYPE@ 00000001800062e0     libsetnotif001.obj
 0002:00001300       ??_C@_0BN@BIBNPHHO@JVMTI_ERROR_ILLEGAL_ARGUMENT@ 0000000180006300     libsetnotif001.obj
 0002:00001320       ??_C@_0BK@KKNDHDCE@JVMTI_ERROR_NATIVE_METHOD@ 0000000180006320     libsetnotif001.obj
 0002:00001340       ??_C@_0BK@PMKCFHAE@JVMTI_ERROR_OUT_OF_MEMORY@ 0000000180006340     libsetnotif001.obj
 0002:00001360       ??_C@_0BK@NNJBDMNB@JVMTI_ERROR_ACCESS_DENIED@ 0000000180006360     libsetnotif001.obj
 0002:00001380       ??_C@_0BI@GHECLMNC@JVMTI_ERROR_WRONG_PHASE@ 0000000180006380     libsetnotif001.obj
 0002:00001398       ??_C@_0BF@OLIHJOII@JVMTI_ERROR_INTERNAL@ 0000000180006398     libsetnotif001.obj
 0002:000013b0       ??_C@_0BO@EOHGKJHI@JVMTI_ERROR_UNATTACHED_THREAD@ 00000001800063b0     libsetnotif001.obj
 0002:000013d0       ??_C@_0CA@LKHFDACL@JVMTI_ERROR_INVALID_ENVIRONMENT@ 00000001800063d0     libsetnotif001.obj
 0002:000013f0       ??_C@_0BA@MMFHLOKK@?$DMunknown?5error?$DO@ 00000001800063f0     libsetnotif001.obj
 0002:00001400       ??_C@_0CF@CBHOKDB@throwable?5?$DN?5jni?9?$DOExceptionOccur@ 0000000180006400     libsetnotif001.obj
 0002:00001428       ??_C@_03OFAPEBGM@?$CFs?6@  0000000180006428     libsetnotif001.obj
 0002:00001430       ??_C@_0DM@LPIGEGNJ@s?2test?2hotspot?2jtreg?2vmTestbase@ 0000000180006430     libsetnotif001.obj
 0002:00001470       ??_C@_0CC@NFCNPEPK@Exception?5in?5JNI?5call?5?$CIcleared?$CJ@ 0000000180006470     libsetnotif001.obj
 0002:00001498       ??_C@_0BJ@IBAKFIKF@jni?9?$DOExceptionDescribe?$CI?$CJ@ 0000000180006498     libsetnotif001.obj
 0002:000014b8       ??_C@_0BG@GGKALKMH@jni?9?$DOExceptionClear?$CI?$CJ@ 00000001800064b8     libsetnotif001.obj
 0002:000014d0       ??_C@_0CF@JMGFGJLJ@?$CD?5?5?5verified?5JNI?5assertion?5is?5F@ 00000001800064d0     libsetnotif001.obj
 0002:000014f8       ??_C@_0CB@MLNJNCLJ@?5?5jvmti?5error?3?5code?$DN?$CFd?0?5name?$DN?$CFs@ 00000001800064f8     libsetnotif001.obj
 0002:00001520       ??_C@_0CD@OHBGDKMK@?$CD?5?5?5jvmti?5error?3?5code?$DN?$CFd?0?5name?$DN@ 0000000180006520     libsetnotif001.obj
 0002:00001548       ??_C@_0CG@JNNCGPHB@?$CD?5?5?5error?5expected?3?5code?$DN?$CFd?0?5na@ 0000000180006548     libsetnotif001.obj
 0002:00001570       ??_C@_0EB@IMGKPCGE@?$CIstr_obj?5?$DN?5jni?9?$DONewStringUTF?$CIco@ 0000000180006570     libsetnotif001.obj
 0002:000015c0       ??_C@_0EA@HFOGGBCC@s?2test?2hotspot?2jtreg?2vmTestbase@ 00000001800065c0     libsetnotif001.obj
 0002:00001600       ??_C@_05KKCIMGE@error@     0000000180006600     libsetnotif001.obj
 0002:00001608       ??_C@_0CJ@JACLEAA@Test?5failed?5by?5setFailStatus?$CI?$CJ?4@ 0000000180006608     libsetnotif001.obj
 0002:00001640       ??_C@_0EA@PNBCDMOA@s?2test?2hotspot?2jtreg?2vmTestbase@ 0000000180006640     libsetnotif001.obj
 0002:00001680       ??_C@_0DI@ILAHDLMP@?$CI?$CKagentThreadProc?$CJ?$CIjvmti_env?0?5a@ 0000000180006680     libsetnotif001.obj
 0002:000016b8       ??_C@_0BD@KDBALNLB@JVMTI?5agent?5thread@ 00000001800066b8     libsetnotif001.obj
 0002:000016d0       ??_C@_0BB@NOKBFPFO@java?1lang?1Thread@ 00000001800066d0     libsetnotif001.obj
 0002:000016e4       ??_C@_06FALKBLGB@?$DMinit?$DO@ 00000001800066e4     libsetnotif001.obj
 0002:000016f0       ??_C@_0BG@IKDDPPGD@?$CILjava?1lang?1String?$DL?$CJV@ 00000001800066f0     libsetnotif001.obj
 0002:00001710       ??_C@_0EB@IFJBFEKC@?$CIthreadClass?5?$DN?5jni_env?9?$DOFindCla@ 0000000180006710     libsetnotif001.obj
 0002:00001760       ??_C@_0GF@FGFIBKKL@?$CIthreadCtor?5?$DN?5jni_env?9?$DOGetMetho@ 0000000180006760     libsetnotif001.obj
 0002:000017c8       ??_C@_0DN@NCPDJLOG@?$CIthreadName?5?$DN?5jni_env?9?$DONewStrin@ 00000001800067c8     libsetnotif001.obj
 0002:00001810       ??_C@_0FE@PFKODBGC@?$CIthreadObject?5?$DN?5jni_env?9?$DONewObj@ 0000000180006810     libsetnotif001.obj
 0002:00001870       ??_C@_0ED@HOBAHHJI@?$CIthreadGlobalRef?5?$DN?5jni_env?9?$DONew@ 0000000180006870     libsetnotif001.obj
 0002:000018c0       ??_C@_0FN@HNJJAHFC@jvmti_env?9?$DORunAgentThread?$CIagent@ 00000001800068c0     libsetnotif001.obj
 0002:00001920       ??_C@_0EA@MOJDNKDF@Debuggee?5status?5sync?5aborted?5be@ 0000000180006920     libsetnotif001.obj
 0002:00001960       ??_C@_0EA@EEOEJAEN@status?5?$DN?5syncDebuggeeStatus?$CIjni@ 0000000180006960     libsetnotif001.obj
 0002:000019a0       ??_C@_0BL@JBCFNBMB@nsk_jvmti_resetAgentData?$CI?$CJ@ 00000001800069a0     libsetnotif001.obj
 0002:000019c0       ??_C@_0EL@LPBEELIP@s?2test?2hotspot?2jtreg?2vmTestbase@ 00000001800069c0     libsetnotif001.obj
 0002:00001a10       ??_C@_0CK@JDAMFDMJ@jvmti?9?$DOSetTag?$CIo?0?5tag?$CJ?5?$DN?$DN?5JVMTI_@ 0000000180006a10     libsetnotif001.obj
 0002:00001a40       ??_C@_0CC@DAMNHKNI@Can?8t?5set?5tag?5?$CFli?5for?5object?5?$CFl@ 0000000180006a40     libsetnotif001.obj
 0002:00001a68       ??_C@_0DL@HAJPNKEF@jvmti?9?$DOGetObjectHashCode?$CIo?0?5?$CGha@ 0000000180006a68     libsetnotif001.obj
 0002:00001aa8       ??_C@_0BL@JFPIEOBF@Can?8t?5get?5hash?5object?5?$CFlx?6@ 0000000180006aa8     libsetnotif001.obj
 0002:00001ac8       ??_C@_0BG@DICPHBKN@setTag?3?5?$CF08x?5?$DM?9?5?$CF?53li@ 0000000180006ac8     libsetnotif001.obj
 0002:00001ae0       ??_C@_0DH@FCEEBDMJ@?$CIs?5?$DN?5jni?9?$DOGetStringUTFChars?$CIsIn@ 0000000180006ae0     libsetnotif001.obj
 0002:00001b18       ??_C@_0BJ@OKKGHDCN@Can?8t?5get?5string?5at?5?$CF?$CDp?6@ 0000000180006b18     libsetnotif001.obj
 0002:00001b38       ??_C@_0BP@EKFLGGFJ@Can?8t?5get?5string?5at?5?$CF?$CDp?3?5null?6@ 0000000180006b38     libsetnotif001.obj
 0002:00001b58       ??_C@_06ICODBHCL@?5?1?1?5?$CFs@ 0000000180006b58     libsetnotif001.obj
 0002:00001b60       ??_C@_0DB@KGFPLEGO@?$CIr?5?$DN?5jvmti?9?$DOGetTag?$CIo?0?5?$CGtag?$CJ?$CJ?5?$DN?$DN@ 0000000180006b60     libsetnotif001.obj
 0002:00001b98       ??_C@_0CO@PDAGBCGJ@Can?8t?5GetTag?5for?5object?5?$CFlx?4?5Re@ 0000000180006b98     libsetnotif001.obj
 0002:00001bc8       ??_C@_0CH@HPEODOHC@TEST_BUG?3?5Max?4?5number?5of?5refs?5r@ 0000000180006bc8     libsetnotif001.obj
 0002:00001bf0       ??_C@_0DI@PHFCABIM@?$CIr?5?$DN?5jvmti?9?$DOGetTag?$CIfrom?0?5?$CGtagFr@ 0000000180006bf0     libsetnotif001.obj
 0002:00001c28       ??_C@_0DI@MDEGFNKD@TEST_BUG?3?5Can?8t?5GetTag?5for?5obje@ 0000000180006c28     libsetnotif001.obj
 0002:00001c60       ??_C@_0DE@MLELJAHM@?$CIr?5?$DN?5jvmti?9?$DOGetTag?$CIto?0?5?$CGtagTo?$CJ?$CJ@ 0000000180006c60     libsetnotif001.obj
 0002:00001c98       ??_C@_0BB@BLBLPJGP@?$DO?$DO?$DO?5catching?5?$CFs?6@ 0000000180006c98     libsetnotif001.obj
 0002:00001cb0       ??_C@_0CN@LEIBHLMB@?$CIRawMonitorEnter?$CJ?5unexpected?5er@ 0000000180006cb0     libsetnotif001.obj
 0002:00001ce0       ??_C@_0DI@GKEOLDMI@Wrong?5notification?3?5event?5?$CFs?5?$CI?$CF@ 0000000180006ce0     libsetnotif001.obj
 0002:00001d18       ??_C@_0CM@BHOJNKDE@?$CIRawMonitorExit?$CJ?5unexpected?5err@ 0000000180006d18     libsetnotif001.obj
 0002:00001d48       ??_C@_0BC@JJNAIJBA@?$DO?$DO?$DO?5disabling?5?$CFs?6@ 0000000180006d48     libsetnotif001.obj
 0002:00001d60       ??_C@_0BN@HOPPFFCI@Fail?5to?5disable?5?$CFs?3?5?$CFs?5?$CI?$CFd?$CJ?6@ 0000000180006d60     libsetnotif001.obj
 0002:00001d80       ??_C@_0BB@KEOFOLHI@?$DO?$DO?$DO?5enabling?5?$CFs?6@ 0000000180006d80     libsetnotif001.obj
 0002:00001d98       ??_C@_0BM@DCBPOLP@Fail?5to?5enable?5?$CFs?3?5?$CFs?5?$CI?$CFd?$CJ?6@ 0000000180006d98     libsetnotif001.obj
 0002:00001db4       ??_C@_04PFANPMCN@?$CII?$CJV@ 0000000180006db4     libsetnotif001.obj
 0002:00001dbc       ??_C@_06MADNOIIM@meth01@   0000000180006dbc     libsetnotif001.obj
 0002:00001dc8       ??_C@_0CB@IKAFJBHN@?$CIGetStaticMethodID?$CJ?5returns?5nul@ 0000000180006dc8     libsetnotif001.obj
 0002:00001df0       ??_C@_0CL@GMOLCHIJ@?$CISetBreakpoint?$CJ?5unexpected?5erro@ 0000000180006df0     libsetnotif001.obj
 0002:00001e1c       ??_C@_01JPJNBJEM@I@        0000000180006e1c     libsetnotif001.obj
 0002:00001e20       ??_C@_03IAKKBENL@fld@      0000000180006e20     libsetnotif001.obj
 0002:00001e28       ??_C@_0DB@ELOCAPIE@?$CISetFieldAccessWatch?$CJ?5unexpecte@ 0000000180006e28     libsetnotif001.obj
 0002:00001e60       ??_C@_0DB@NFHHHHOJ@Warning?3?5SetFieldAccessWatch?5is@ 0000000180006e60     libsetnotif001.obj
 0002:00001e98       ??_C@_0DH@EFJMOCPE@?$CISetFieldModificationWatch?$CJ?5une@ 0000000180006e98     libsetnotif001.obj
 0002:00001ed0       ??_C@_0DH@KCGKHHKP@Warning?3?5SetFieldModificationWa@ 0000000180006ed0     libsetnotif001.obj
 0002:00001f08       ??_C@_0M@KABMGAEH@?$DO?$DO?$DO?5VMInit?6@ 0000000180006f08     libsetnotif001.obj
 0002:00001f18       ??_C@_0CM@JDNNOJJD@?$CIIsMethodNative?$CJ?5unexpected?5err@ 0000000180006f18     libsetnotif001.obj
 0002:00001f48       ??_C@_0CM@DJHCDKC@?$CINotifyFramePop?$CJ?5unexpected?5err@ 0000000180006f48     libsetnotif001.obj
 0002:00001f78       ??_C@_09OPJEJKBL@printdump@ 0000000180006f78     libsetnotif001.obj
 0002:00001f88       ??_C@_0CK@DEFLIKCM@Wrong?5result?5of?5a?5valid?5call?5to@ 0000000180006f88     libsetnotif001.obj
 0002:00001fb8       ??_C@_0DG@LAJPGIIE@?$CIGetPotentialCapabilities?$CJ?5unex@ 0000000180006fb8     libsetnotif001.obj
 0002:00001ff0       ??_C@_0CN@LKPEOJPO@?$CIAddCapabilities?$CJ?5unexpected?5er@ 0000000180006ff0     libsetnotif001.obj
 0002:00002020       ??_C@_0CN@BCCBOHCH@?$CIGetCapabilities?$CJ?5unexpected?5er@ 0000000180007020     libsetnotif001.obj
 0002:00002050       ??_C@_0N@HJAMKMBE@_access_lock@ 0000000180007050     libsetnotif001.obj
 0002:00002060       ??_C@_0CO@BLGNGBDG@?$CICreateRawMonitor?$CJ?5unexpected?5e@ 0000000180007060     libsetnotif001.obj
 0002:00002090       ??_C@_0CP@IMINGNLL@?$CISetEventCallbacks?$CJ?5unexpected?5@ 0000000180007090     libsetnotif001.obj
 0002:000020c0       ??_C@_0CA@HMHAPBAI@No?5notification?3?5event?5?$CFs?5?$CI?$CFd?$CJ?6@ 00000001800070c0     libsetnotif001.obj
 0002:000020e0       ??_C@_0CA@JIHPCMLD@?$DO?$DO?$DO?5?$CFs?5?$CI?$CFd?$CJ?0?5notifications?3?5?$CFd?6@ 00000001800070e0     libsetnotif001.obj
 0002:00002110       ??_C@_1EC@JIJBPKFM@?$AAa?$AAp?$AAi?$AA?9?$AAm?$AAs?$AA?9?$AAw?$AAi?$AAn?$AA?9?$AAc?$AAo?$AAr?$AAe@ 0000000180007110     MSVCRT:thread_safe_statics.obj
 0002:00002158       ??_C@_1BK@MGMFAEKH@?$AAk?$AAe?$AAr?$AAn?$AAe?$AAl?$AA3?$AA2?$AA?4?$AAd?$AAl?$AAl@ 0000000180007158     MSVCRT:thread_safe_statics.obj
 0002:00002178       ??_C@_0BJ@JEBJOJFJ@SleepConditionVariableCS@ 0000000180007178     MSVCRT:thread_safe_statics.obj
 0002:00002198       ??_C@_0BJ@PGPPEPCC@WakeAllConditionVariable@ 0000000180007198     MSVCRT:thread_safe_statics.obj
 0002:000021b8       _pDefaultRawDllMain        00000001800071b8     MSVCRT:dll_dllmain.obj
 0002:000021b8       _pRawDllMain               00000001800071b8     MSVCRT:dll_dllmain.obj
 0002:000021c0       __xmm@ffffffffffffffffffffffffffffffff 00000001800071c0     MSVCRT:utility.obj
 0002:000021d0       _load_config_used          00000001800071d0     MSVCRT:loadcfg.obj
 0002:00002380       _tls_used                  0000000180007380     MSVCRT:tlssup.obj
 0002:000023a8       __volatile_metadata        00000001800073a8     <linker-defined>
 0002:00002768       __rtc_iaa                  0000000180007768     MSVCRT:initsect.obj
 0002:00002770       __rtc_izz                  0000000180007770     MSVCRT:initsect.obj
 0002:00002778       __rtc_taa                  0000000180007778     MSVCRT:initsect.obj
 0002:00002780       __rtc_tzz                  0000000180007780     MSVCRT:initsect.obj
 0002:00002788       _tls_start                 0000000180007788     MSVCRT:tlssup.obj
 0002:0000278c       _Init_thread_epoch         000000018000778c     MSVCRT:thread_safe_statics.obj
 0002:00002790       _tls_end                   0000000180007790     MSVCRT:tlssup.obj
 0002:00002ea0       __IMPORT_DESCRIPTOR_KERNEL32 0000000180007ea0     kernel32:KERNEL32.dll
 0002:00002eb4       __IMPORT_DESCRIPTOR_VCRUNTIME140 0000000180007eb4     vcruntime:VCRUNTIME140.dll
 0002:00002ec8       __IMPORT_DESCRIPTOR_api-ms-win-crt-runtime-l1-1-0 0000000180007ec8     ucrt:api-ms-win-crt-runtime-l1-1-0.dll
 0002:00002edc       __IMPORT_DESCRIPTOR_api-ms-win-crt-stdio-l1-1-0 0000000180007edc     ucrt:api-ms-win-crt-stdio-l1-1-0.dll
 0002:00002ef0       __IMPORT_DESCRIPTOR_api-ms-win-crt-string-l1-1-0 0000000180007ef0     ucrt:api-ms-win-crt-string-l1-1-0.dll
 0002:00002f04       __NULL_IMPORT_DESCRIPTOR   0000000180007f04     kernel32:KERNEL32.dll
 0003:00000030       _Init_global_epoch         0000000180009030     MSVCRT:thread_safe_statics.obj
 0003:00000040       __security_cookie          0000000180009040     MSVCRT:gs_cookie.obj
 0003:00000048       __security_cookie_complement 0000000180009048     MSVCRT:gs_cookie.obj
 0003:00000050       __scrt_native_dllmain_reason 0000000180009050     MSVCRT:utility.obj
 0003:00000058       __isa_available            0000000180009058     MSVCRT:cpu_disp.obj
 0003:0000005c       __isa_enabled              000000018000905c     MSVCRT:cpu_disp.obj
 0003:00000060       __memset_fast_string_threshold 0000000180009060     MSVCRT:cpu_disp.obj
 0003:00000068       __memset_nt_threshold      0000000180009068     MSVCRT:cpu_disp.obj
 0003:00000070       __scrt_ucrt_dll_is_in_use  0000000180009070     MSVCRT:ucrt_stubs.obj
 0003:00000080       g_wrongHeapCallbacks       0000000180009080     libsetnotif001.obj
 0003:00000100       g_szTagInfo                0000000180009100     libsetnotif001.obj
 0003:00002040       g_tagFlags                 000000018000b040     libsetnotif001.obj
 0003:00002428       g_refsToVerifyCnt          000000018000b428     libsetnotif001.obj
 0003:0000242c       g_fakeUserData             000000018000b42c     libsetnotif001.obj
 0003:00002430       g_tagVisitCount            000000018000b430     libsetnotif001.obj
 0003:000033d0       g_refsToVerify             000000018000c3d0     libsetnotif001.obj
 0003:0001aad0       g_userDataError            0000000180023ad0     libsetnotif001.obj
 0003:0001ae90       ?_OptionsStorage@?1??__local_stdio_printf_options@@9@4_KA 0000000180023e90     libsetnotif001.obj
 0003:0001b458       _tls_index                 0000000180024458     MSVCRT:tlssup.obj
 0003:0001b460       __scrt_current_native_startup_state 0000000180024460     MSVCRT:utility.obj
 0003:0001b468       __scrt_native_startup_lock 0000000180024468     MSVCRT:utility.obj
 0003:0001b4a8       __scrt_debugger_hook_flag  00000001800244a8     MSVCRT:utility_desktop.obj
 0003:0001b4b0       ?__type_info_root_node@@3U__type_info_node@@A 00000001800244b0     MSVCRT:tncleanup.obj
 0003:0001b4c0       ?_OptionsStorage@?1??__local_stdio_scanf_options@@9@4_KA 00000001800244c0     MSVCRT:default_local_stdio_options.obj
 0003:0001b4c8       __favor                    00000001800244c8     MSVCRT:cpu_disp.obj
 0003:0001b4d0       __dyn_tls_init_callback    00000001800244d0     <common>

 entry point at        0001:00002dc0

 Static symbols

 0000:fffd9000       .debug$S                   0000000180000000     setnotif001.exp
 0000:fffd9000       .debug$S                   0000000180000000     vcruntime:VCRUNTIME140.dll
 0000:fffd9000       .debug$S                   0000000180000000     vcruntime:VCRUNTIME140.dll
 0000:fffd9000       .debug$S                   0000000180000000     vcruntime:VCRUNTIME140.dll
 0000:fffd9000       .debug$S                   0000000180000000     vcruntime:VCRUNTIME140.dll
 0000:fffd9000       .debug$S                   0000000180000000     vcruntime:VCRUNTIME140.dll
 0000:fffd9000       .debug$S                   0000000180000000     vcruntime:VCRUNTIME140.dll
 0000:fffd9000       .debug$S                   0000000180000000     vcruntime:VCRUNTIME140.dll
 0000:fffd9000       .debug$S                   0000000180000000     ucrt:api-ms-win-crt-convert-l1-1-0.dll
 0002:ffffb000       .idata$6                   0000000180000000     ucrt:api-ms-win-crt-convert-l1-1-0.dll
 0000:fffd9000       .debug$S                   0000000180000000     ucrt:api-ms-win-crt-heap-l1-1-0.dll
 0000:fffd9000       .debug$S                   0000000180000000     ucrt:api-ms-win-crt-heap-l1-1-0.dll
 0000:fffd9000       .debug$S                   0000000180000000     ucrt:api-ms-win-crt-heap-l1-1-0.dll
 0000:fffd9000       .debug$S                   0000000180000000     ucrt:api-ms-win-crt-heap-l1-1-0.dll
 0002:ffffb000       .idata$6                   0000000180000000     ucrt:api-ms-win-crt-heap-l1-1-0.dll
 0000:fffd9000       .debug$S                   0000000180000000     ucrt:api-ms-win-crt-runtime-l1-1-0.dll
 0000:fffd9000       .debug$S                   0000000180000000     ucrt:api-ms-win-crt-runtime-l1-1-0.dll
 0000:fffd9000       .debug$S                   0000000180000000     ucrt:api-ms-win-crt-runtime-l1-1-0.dll
 0000:fffd9000       .debug$S                   0000000180000000     ucrt:api-ms-win-crt-runtime-l1-1-0.dll
 0000:fffd9000       .debug$S                   0000000180000000     ucrt:api-ms-win-crt-runtime-l1-1-0.dll
 0000:fffd9000       .debug$S                   0000000180000000     ucrt:api-ms-win-crt-runtime-l1-1-0.dll
 0000:fffd9000       .debug$S                   0000000180000000     ucrt:api-ms-win-crt-runtime-l1-1-0.dll
 0000:fffd9000       .debug$S                   0000000180000000     ucrt:api-ms-win-crt-runtime-l1-1-0.dll
 0000:fffd9000       .debug$S                   0000000180000000     ucrt:api-ms-win-crt-runtime-l1-1-0.dll
 0000:fffd9000       .debug$S                   0000000180000000     ucrt:api-ms-win-crt-runtime-l1-1-0.dll
 0000:fffd9000       .debug$S                   0000000180000000     ucrt:api-ms-win-crt-runtime-l1-1-0.dll
 0000:fffd9000       .debug$S                   0000000180000000     ucrt:api-ms-win-crt-runtime-l1-1-0.dll
 0000:fffd9000       .debug$S                   0000000180000000     ucrt:api-ms-win-crt-runtime-l1-1-0.dll
 0000:fffd9000       .debug$S                   0000000180000000     ucrt:api-ms-win-crt-runtime-l1-1-0.dll
 0000:fffd9000       .debug$S                   0000000180000000     ucrt:api-ms-win-crt-runtime-l1-1-0.dll
 0000:fffd9000       .debug$S                   0000000180000000     ucrt:api-ms-win-crt-runtime-l1-1-0.dll
 0000:fffd9000       .debug$S                   0000000180000000     ucrt:api-ms-win-crt-stdio-l1-1-0.dll
 0000:fffd9000       .debug$S                   0000000180000000     ucrt:api-ms-win-crt-stdio-l1-1-0.dll
 0000:fffd9000       .debug$S                   0000000180000000     ucrt:api-ms-win-crt-stdio-l1-1-0.dll
 0000:fffd9000       .debug$S                   0000000180000000     ucrt:api-ms-win-crt-stdio-l1-1-0.dll
 0000:fffd9000       .debug$S                   0000000180000000     ucrt:api-ms-win-crt-stdio-l1-1-0.dll
 0000:fffd9000       .debug$S                   0000000180000000     ucrt:api-ms-win-crt-stdio-l1-1-0.dll
 0000:fffd9000       .debug$S                   0000000180000000     ucrt:api-ms-win-crt-stdio-l1-1-0.dll
 0000:fffd9000       .debug$S                   0000000180000000     ucrt:api-ms-win-crt-stdio-l1-1-0.dll
 0000:fffd9000       .debug$S                   0000000180000000     ucrt:api-ms-win-crt-stdio-l1-1-0.dll
 0000:fffd9000       .debug$S                   0000000180000000     ucrt:api-ms-win-crt-stdio-l1-1-0.dll
 0000:fffd9000       .debug$S                   0000000180000000     ucrt:api-ms-win-crt-string-l1-1-0.dll
 0000:fffd9000       .debug$S                   0000000180000000     ucrt:api-ms-win-crt-string-l1-1-0.dll
 0000:fffd9000       .debug$S                   0000000180000000     ucrt:api-ms-win-crt-string-l1-1-0.dll
 0000:fffd9000       .debug$S                   0000000180000000     ucrt:api-ms-win-crt-string-l1-1-0.dll
 0000:fffd9000       .debug$S                   0000000180000000     ucrt:api-ms-win-crt-string-l1-1-0.dll
 0000:fffd9000       .debug$S                   0000000180000000     ucrt:api-ms-win-crt-string-l1-1-0.dll
 0000:fffd9000       .debug$S                   0000000180000000     ucrt:api-ms-win-crt-string-l1-1-0.dll
 0000:fffd9000       .debug$S                   0000000180000000     ucrt:api-ms-win-crt-string-l1-1-0.dll
 0000:fffd9000       .debug$S                   0000000180000000     kernel32:KERNEL32.dll
 0000:fffd9000       .debug$S                   0000000180000000     kernel32:KERNEL32.dll
 0000:fffd9000       .debug$S                   0000000180000000     kernel32:KERNEL32.dll
 0000:fffd9000       .debug$S                   0000000180000000     kernel32:KERNEL32.dll
 0000:fffd9000       .debug$S                   0000000180000000     kernel32:KERNEL32.dll
 0000:fffd9000       .debug$S                   0000000180000000     kernel32:KERNEL32.dll
 0000:fffd9000       .debug$S                   0000000180000000     kernel32:KERNEL32.dll
 0000:fffd9000       .debug$S                   0000000180000000     kernel32:KERNEL32.dll
 0000:fffd9000       .debug$S                   0000000180000000     kernel32:KERNEL32.dll
 0000:fffd9000       .debug$S                   0000000180000000     kernel32:KERNEL32.dll
 0000:fffd9000       .debug$S                   0000000180000000     kernel32:KERNEL32.dll
 0000:fffd9000       .debug$S                   0000000180000000     kernel32:KERNEL32.dll
 0000:fffd9000       .debug$S                   0000000180000000     kernel32:KERNEL32.dll
 0000:fffd9000       .debug$S                   0000000180000000     kernel32:KERNEL32.dll
 0000:fffd9000       .debug$S                   0000000180000000     kernel32:KERNEL32.dll
 0000:fffd9000       .debug$S                   0000000180000000     kernel32:KERNEL32.dll
 0000:fffd9000       .debug$S                   0000000180000000     kernel32:KERNEL32.dll
 0000:fffd9000       .debug$S                   0000000180000000     kernel32:KERNEL32.dll
 0000:fffd9000       .debug$S                   0000000180000000     kernel32:KERNEL32.dll
 0000:fffd9000       .debug$S                   0000000180000000     kernel32:KERNEL32.dll
 0000:fffd9000       .debug$S                   0000000180000000     kernel32:KERNEL32.dll
 0000:fffd9000       .debug$S                   0000000180000000     kernel32:KERNEL32.dll
 0000:fffd9000       .debug$S                   0000000180000000     kernel32:KERNEL32.dll
 0000:fffd9000       .debug$S                   0000000180000000     kernel32:KERNEL32.dll
 0000:fffd9000       .debug$S                   0000000180000000     kernel32:KERNEL32.dll
 0000:fffd9000       .debug$S                   0000000180000000     kernel32:KERNEL32.dll
 0000:fffd9000       .debug$S                   0000000180000000     kernel32:KERNEL32.dll
 0000:fffd9000       .debug$S                   0000000180000000     kernel32:KERNEL32.dll
 0001:0000156c       addRefToVerify             000000018000256c f   libsetnotif001.obj
 0001:000015d8       agentThreadWrapper         00000001800025d8 f   libsetnotif001.obj
 0001:00001978       file_basename              0000000180002978 f   libsetnotif001.obj
 0001:000022a8       startAgentThreadWrapper    00000001800032a8 f   libsetnotif001.obj
 0001:000025e8       syncDebuggeeStatus         00000001800035e8 f   libsetnotif001.obj
 0001:00002888       capture_previous_context   0000000180003888 f   MSVCRT:gs_report.obj
 0001:000028fc       ?__scrt_initialize_thread_safe_statics@@YAHXZ 00000001800038fc f   MSVCRT:thread_safe_statics.obj
 0001:000029cc       ?__scrt_uninitialize_thread_safe_statics@@YAXXZ 00000001800039cc f   MSVCRT:thread_safe_statics.obj
 0001:00002a70       $$000000                   0000000180003a70     MSVCRT:amdsecgs.obj
 0001:00002aa0       ?dllmain_crt_dispatch@@YAHQEAUHINSTANCE__@@KQEAX@Z 0000000180003aa0 f   MSVCRT:dll_dllmain.obj
 0001:00002af0       ?dllmain_crt_process_attach@@YAHQEAUHINSTANCE__@@QEAX@Z 0000000180003af0 f   MSVCRT:dll_dllmain.obj
 0001:00002c08       ?dllmain_crt_process_detach@@YAH_N@Z 0000000180003c08 f   MSVCRT:dll_dllmain.obj
 0001:00002c8c       ?dllmain_dispatch@@YAHQEAUHINSTANCE__@@KQEAX@Z 0000000180003c8c f   MSVCRT:dll_dllmain.obj
 0001:000036a0       $$000000                   00000001800046a0     MSVCRT:guard_dispatch.obj
 0001:000036c0       $$000000                   00000001800046c0     MSVCRT:guard_xfg_dispatch.obj
 0001:000036d6       ?fin$0@?0??dllmain_crt_process_attach@@YAHQEAUHINSTANCE__@@QEAX@Z@4HA 00000001800046d6 f   MSVCRT:dll_dllmain.obj
 0001:000036ed       ?fin$0@?0??dllmain_crt_process_detach@@YAH_N@Z@4HA 00000001800046ed f   MSVCRT:dll_dllmain.obj
 0001:00003706       ?fin$1@?0??dllmain_crt_process_detach@@YAH_N@Z@4HA 0000000180004706 f   MSVCRT:dll_dllmain.obj
 0001:0000371a       ?filt$0@?0??dllmain_dispatch@@YAHQEAUHINSTANCE__@@KQEAX@Z@4HA 000000018000471a f   MSVCRT:dll_dllmain.obj
 0001:00003750       __scrt_is_nonwritable_in_current_image$filt$0 0000000180004750 f   MSVCRT:utility.obj
 0002:000001e8       ?__scrt_initialize_tss_var@@3P6AHXZEA 00000001800051e8     MSVCRT:thread_safe_statics.obj
 0002:00000310       ?opcLengths@@3QBEB         0000000180005310     libsetnotif001.obj
 0002:00002100       GS_ExceptionPointers       0000000180007100     MSVCRT:gs_report.obj
 0002:00002798       $unwind$fprintf            0000000180007798     libsetnotif001.obj
 0002:000027a4       $unwind$printf             00000001800077a4     libsetnotif001.obj
 0002:000027b0       $unwind$?NewObject@JNIEnv_@@QEAAPEAV_jobject@@PEAV_jclass@@PEAU_jmethodID@@ZZ 00000001800077b0     libsetnotif001.obj
 0002:000027b0       $unwind$nsk_lcomplain      00000001800077b0     libsetnotif001.obj
 0002:000027b0       $unwind$nsk_ldisplay       00000001800077b0     libsetnotif001.obj
 0002:000027b8       $unwind$Java_nsk_jvmti_SetEventNotificationMode_setnotif001_enableEv 00000001800077b8     libsetnotif001.obj
 0002:000027b8       $unwind$nsk_lvdisplay      00000001800077b8     libsetnotif001.obj
 0002:000027b8       $unwind$_RTC_Initialize    00000001800077b8     MSVCRT:initsect.obj
 0002:000027b8       $unwind$_RTC_Terminate     00000001800077b8     MSVCRT:initsect.obj
 0002:000027b8       $unwind$?__scrt_initialize_thread_safe_statics@@YAHXZ 00000001800077b8     MSVCRT:thread_safe_statics.obj
 0002:000027c4       $unwind$nsk_lvcomplain     00000001800077c4     libsetnotif001.obj
 0002:000027dc       $unwind$nsk_ltrace         00000001800077dc     libsetnotif001.obj
 0002:000027dc       $unwind$__report_gsfailure 00000001800077dc     MSVCRT:gs_report.obj
 0002:000027e4       $unwind$MethodExit         00000001800077e4     libsetnotif001.obj
 0002:000027e4       $unwind$SingleStep         00000001800077e4     libsetnotif001.obj
 0002:000027e4       $unwind$VMInit             00000001800077e4     libsetnotif001.obj
 0002:000027e4       $unwind$nsk_lvtrace        00000001800077e4     libsetnotif001.obj
 0002:000027e4       $unwind$__raise_securityfailure 00000001800077e4     MSVCRT:gs_report.obj
 0002:000027e4       $unwind$__scrt_initialize_crt 00000001800077e4     MSVCRT:utility.obj
 0002:000027e4       $unwind$__scrt_initialize_onexit_tables 00000001800077e4     MSVCRT:utility.obj
 0002:000027e4       $unwind$__scrt_release_startup_lock 00000001800077e4     MSVCRT:utility.obj
 0002:000027e4       $unwind$__scrt_uninitialize_crt 00000001800077e4     MSVCRT:utility.obj
 0002:000027e4       $unwind$_onexit            00000001800077e4     MSVCRT:utility.obj
 0002:000027ec       $unwind$nsk_lverify        00000001800077ec     libsetnotif001.obj
 0002:000027fc       $unwind$nsk_vprintf        00000001800077fc     libsetnotif001.obj
 0002:0000280c       $unwind$nsk_printf         000000018000780c     libsetnotif001.obj
 0002:00002814       $unwind$?nsk_jni_lverify@@YAHHPEAUJNIEnv_@@HQEBDH1ZZ 0000000180007814     libsetnotif001.obj
 0002:00002828       $unwind$?nsk_jni_check_exception@@YAHPEAUJNIEnv_@@QEBDH@Z 0000000180007828     libsetnotif001.obj
 0002:00002844       $unwind$Breakpoint         0000000180007844     libsetnotif001.obj
 0002:00002844       $unwind$ClassLoad          0000000180007844     libsetnotif001.obj
 0002:00002844       $unwind$ClassPrepare       0000000180007844     libsetnotif001.obj
 0002:00002844       $unwind$Exception          0000000180007844     libsetnotif001.obj
 0002:00002844       $unwind$ExceptionCatch     0000000180007844     libsetnotif001.obj
 0002:00002844       $unwind$FieldAccess        0000000180007844     libsetnotif001.obj
 0002:00002844       $unwind$FieldModification  0000000180007844     libsetnotif001.obj
 0002:00002844       $unwind$FramePop           0000000180007844     libsetnotif001.obj
 0002:00002844       $unwind$Java_nsk_jvmti_unit_FollowReferences_FollowRefObjects_resetTags 0000000180007844     libsetnotif001.obj
 0002:00002844       $unwind$ThreadEnd          0000000180007844     libsetnotif001.obj
 0002:00002844       $unwind$ThreadStart        0000000180007844     libsetnotif001.obj
 0002:00002844       $unwind$addRefToVerify     0000000180007844     libsetnotif001.obj
 0002:00002844       $unwind$nsk_jvmti_resetAgentData 0000000180007844     libsetnotif001.obj
 0002:00002844       $unwind$nsk_jvmti_setFailStatus 0000000180007844     libsetnotif001.obj
 0002:00002844       $unwind$__scrt_initialize_default_local_stdio_options 0000000180007844     MSVCRT:default_local_stdio_options.obj
 0002:00002844       $unwind$?dllmain_crt_dispatch@@YAHQEAUHINSTANCE__@@KQEAX@Z 0000000180007844     MSVCRT:dll_dllmain.obj
 0002:00002844       $unwind$DllMain            0000000180007844     MSVCRT:dll_dllmain_stub.obj
 0002:00002844       $unwind$__GSHandlerCheck   0000000180007844     MSVCRT:gshandler.obj
 0002:00002844       $unwind$?__scrt_uninitialize_thread_safe_statics@@YAXXZ 0000000180007844     MSVCRT:thread_safe_statics.obj
 0002:00002844       $unwind$__scrt_acquire_startup_lock 0000000180007844     MSVCRT:utility.obj
 0002:00002844       $unwind$__scrt_dllmain_after_initialize_c 0000000180007844     MSVCRT:utility.obj
 0002:00002844       $unwind$__scrt_dllmain_before_initialize_c 0000000180007844     MSVCRT:utility.obj
 0002:00002844       $unwind$__scrt_dllmain_crt_thread_attach 0000000180007844     MSVCRT:utility.obj
 0002:00002844       $unwind$__scrt_dllmain_crt_thread_detach 0000000180007844     MSVCRT:utility.obj
 0002:00002844       $unwind$__scrt_dllmain_uninitialize_c 0000000180007844     MSVCRT:utility.obj
 0002:00002844       $unwind$__scrt_dllmain_uninitialize_critical 0000000180007844     MSVCRT:utility.obj
 0002:00002844       $unwind$atexit             0000000180007844     MSVCRT:utility.obj
 0002:0000284c       $unwind$nsk_jvmti_lverify  000000018000784c     libsetnotif001.obj
 0002:00002860       $unwind$exitOnError        0000000180007860     libsetnotif001.obj
 0002:00002870       $unwind$Java_nsk_share_jvmti_ArgumentHandler_getAgentOptionsString 0000000180007870     libsetnotif001.obj
 0002:00002884       $unwind$Java_nsk_jvmti_unit_FollowReferences_FollowRefObjects_getTag 0000000180007884     libsetnotif001.obj
 0002:00002884       $unwind$Java_nsk_share_jvmti_DebugeeClass_checkStatus 0000000180007884     libsetnotif001.obj
 0002:00002884       $unwind$agentThreadWrapper 0000000180007884     libsetnotif001.obj
 0002:00002894       $unwind$startAgentThreadWrapper 0000000180007894     libsetnotif001.obj
 0002:000028b0       $unwind$Java_nsk_jvmti_SetEventNotificationMode_setnotif001_getRes 00000001800078b0     libsetnotif001.obj
 0002:000028b0       $unwind$enable             00000001800078b0     libsetnotif001.obj
 0002:000028b0       $unwind$syncDebuggeeStatus 00000001800078b0     libsetnotif001.obj
 0002:000028b0       $unwind$__scrt_dllmain_exception_filter 00000001800078b0     MSVCRT:utility.obj
 0002:000028c4       $unwind$Java_nsk_share_jvmti_DebugeeClass_resetAgentData 00000001800078c4     libsetnotif001.obj
 0002:000028cc       $unwind$MA_checkStatus     00000001800078cc     libsetnotif001.obj
 0002:000028e0       $unwind$Java_nsk_jvmti_unit_FollowReferences_FollowRefObjects_setTag 00000001800078e0     libsetnotif001.obj
 0002:000028f8       $unwind$Java_nsk_jvmti_unit_FollowReferences_FollowRefObjects_addRefToVerify 00000001800078f8     libsetnotif001.obj
 0002:00002914       $unwind$Agent_Initialize   0000000180007914     libsetnotif001.obj
 0002:00002920       $unwind$mark               0000000180007920     libsetnotif001.obj
 0002:00002934       $unwind$disable            0000000180007934     libsetnotif001.obj
 0002:00002934       $unwind$_DllMainCRTStartup 0000000180007934     MSVCRT:dll_dllmain.obj
 0002:00002944       $unwind$setWatches         0000000180007944     libsetnotif001.obj
 0002:00002958       $unwind$MethodEntry        0000000180007958     libsetnotif001.obj
 0002:0000296c       $unwind$capture_previous_context 000000018000796c     MSVCRT:gs_report.obj
 0002:00002978       $unwind$__GSHandlerCheckCommon 0000000180007978     MSVCRT:gshandler.obj
 0002:00002980       $xdatasym                  0000000180007980     MSVCRT:amdsecgs.obj
 0002:00002984       $unwind$?dllmain_crt_process_attach@@YAHQEAUHINSTANCE__@@QEAX@Z 0000000180007984     MSVCRT:dll_dllmain.obj
 0002:000029c0       $unwind$?fin$0@?0??dllmain_crt_process_attach@@YAHQEAUHINSTANCE__@@QEAX@Z@4HA 00000001800079c0     MSVCRT:dll_dllmain.obj
 0002:000029c0       $unwind$?fin$0@?0??dllmain_crt_process_detach@@YAH_N@Z@4HA 00000001800079c0     MSVCRT:dll_dllmain.obj
 0002:000029c0       $unwind$?fin$1@?0??dllmain_crt_process_detach@@YAH_N@Z@4HA 00000001800079c0     MSVCRT:dll_dllmain.obj
 0002:000029c8       $unwind$?dllmain_crt_process_detach@@YAH_N@Z 00000001800079c8     MSVCRT:dll_dllmain.obj
 0002:00002a1c       $unwind$?dllmain_dispatch@@YAHQEAUHINSTANCE__@@KQEAX@Z 0000000180007a1c     MSVCRT:dll_dllmain.obj
 0002:00002a44       $unwind$?filt$0@?0??dllmain_dispatch@@YAHQEAUHINSTANCE__@@KQEAX@Z@4HA 0000000180007a44     MSVCRT:dll_dllmain.obj
 0002:00002a4c       $unwind$__scrt_is_nonwritable_in_current_image 0000000180007a4c     MSVCRT:utility.obj
 0002:00002a6c       $unwind$__scrt_is_nonwritable_in_current_image$filt$0 0000000180007a6c     MSVCRT:utility.obj
 0002:00002a74       $unwind$__scrt_fastfail    0000000180007a74     MSVCRT:utility_desktop.obj
 0002:00002a84       $unwind$__security_init_cookie 0000000180007a84     MSVCRT:gs_support.obj
 0002:00002a90       $unwind$__isa_available_init 0000000180007a90     MSVCRT:cpu_disp.obj
 0002:00002aa0       $xdatasym                  0000000180007aa0     MSVCRT:guard_dispatch.obj
 0002:00002aa8       $xdatasym                  0000000180007aa8     MSVCRT:guard_xfg_dispatch.obj
 0002:00002ab0       .edata                     0000000180007ab0     setnotif001.exp
 0002:00002ad8       rgpv                       0000000180007ad8     setnotif001.exp
 0002:00002b18       rgszName                   0000000180007b18     setnotif001.exp
 0002:00002b58       rgwOrd                     0000000180007b58     setnotif001.exp
 0002:00002b78       szName                     0000000180007b78     setnotif001.exp
 0002:00002b88       $N00001                    0000000180007b88     setnotif001.exp
 0002:00002b97       $N00002                    0000000180007b97     setnotif001.exp
 0002:00002ba4       $N00003                    0000000180007ba4     setnotif001.exp
 0002:00002be1       $N00004                    0000000180007be1     setnotif001.exp
 0002:00002c1c       $N00005                    0000000180007c1c     setnotif001.exp
 0002:00002c61       $N00006                    0000000180007c61     setnotif001.exp
 0002:00002c9e       $N00007                    0000000180007c9e     setnotif001.exp
 0002:00002ce6       $N00008                    0000000180007ce6     setnotif001.exp
 0002:00002d26       $N00009                    0000000180007d26     setnotif001.exp
 0002:00002d63       $N00010                    0000000180007d63     setnotif001.exp
 0002:00002d9e       $N00011                    0000000180007d9e     setnotif001.exp
 0002:00002dcc       $N00012                    0000000180007dcc     setnotif001.exp
 0002:00002dfd       $N00013                    0000000180007dfd     setnotif001.exp
 0002:00002e2c       $N00014                    0000000180007e2c     setnotif001.exp
 0002:00002e5b       $N00015                    0000000180007e5b     setnotif001.exp
 0002:00002e90       $N00016                    0000000180007e90     setnotif001.exp
 0002:0000329a       .idata$6                   000000018000829a     kernel32:KERNEL32.dll
 0002:000032fe       .idata$6                   00000001800082fe     vcruntime:VCRUNTIME140.dll
 0002:0000346a       .idata$6                   000000018000846a     ucrt:api-ms-win-crt-runtime-l1-1-0.dll
 0002:0000348c       .idata$6                   000000018000848c     ucrt:api-ms-win-crt-stdio-l1-1-0.dll
 0002:000034ac       .idata$6                   00000001800084ac     ucrt:api-ms-win-crt-string-l1-1-0.dll
 0003:00000000       ?codeAttributeName@@3PEBDEB 0000000180009000     libsetnotif001.obj
 0003:00000008       ?lineNumberAttributeName@@3PEBDEB 0000000180009008     libsetnotif001.obj
 0003:00000010       ?localVarAttributeName@@3PEBDEB 0000000180009010     libsetnotif001.obj
 0003:00000018       ?localVarTypeAttributeName@@3PEBDEB 0000000180009018     libsetnotif001.obj
 0003:00000020       ?stackMapAttributeName@@3PEBDEB 0000000180009020     libsetnotif001.obj
 0003:00000028       ?callBytes@@3PAEA          0000000180009028     libsetnotif001.obj
 0003:0000002c       ?allocBytes@@3PAEA         000000018000902c     libsetnotif001.obj
 0003:0001aad4       redefineAttempted          0000000180023ad4     libsetnotif001.obj
 0003:0001aad8       nsk_context                0000000180023ad8     libsetnotif001.obj
 0003:0001aae4       redefineSucceed            0000000180023ae4     libsetnotif001.obj
 0003:0001aae8       agentFailed                0000000180023ae8     libsetnotif001.obj
 0003:0001aaec       currentAgentStatus         0000000180023aec     libsetnotif001.obj
 0003:0001aaf0       context                    0000000180023af0     libsetnotif001.obj
 0003:0001aba8       agentThread                0000000180023ba8     libsetnotif001.obj
 0003:0001abb0       agentThreadProc            0000000180023bb0     libsetnotif001.obj
 0003:0001abb8       agentThreadArg             0000000180023bb8     libsetnotif001.obj
 0003:0001abc0       agent_data                 0000000180023bc0     libsetnotif001.obj
 0003:0001abd0       jvmti_env                  0000000180023bd0     libsetnotif001.obj
 0003:0001abd8       jvm                        0000000180023bd8     libsetnotif001.obj
 0003:0001abe0       jni_env                    0000000180023be0     libsetnotif001.obj
 0003:0001abe8       checkStatus_func           0000000180023be8     libsetnotif001.obj
 0003:0001abf0       ?codeAttributeIndex@@3GA   0000000180023bf0     libsetnotif001.obj
 0003:0001abf2       printdump                  0000000180023bf2     libsetnotif001.obj
 0003:0001abf4       ?lineNumberAttributeIndex@@3GA 0000000180023bf4     libsetnotif001.obj
 0003:0001abf8       ?localVarAttributeIndex@@3GA 0000000180023bf8     libsetnotif001.obj
 0003:0001abfc       ?localVarTypeAttributeIndex@@3GA 0000000180023bfc     libsetnotif001.obj
 0003:0001ac00       ?stackMapAttributeIndex@@3GA 0000000180023c00     libsetnotif001.obj
 0003:0001ac04       ?stackFrameOffset@@3GA     0000000180023c04     libsetnotif001.obj
 0003:0001ac08       ?mode@@3HA                 0000000180023c08     libsetnotif001.obj
 0003:0001ac0c       ?constantPoolSize@@3GA     0000000180023c0c     libsetnotif001.obj
 0003:0001ac10       ?orig@@3PEBEEB             0000000180023c10     libsetnotif001.obj
 0003:0001ac18       ?gen@@3PEAEEA              0000000180023c18     libsetnotif001.obj
 0003:0001ac20       ?inputPos@@3PEAEEA         0000000180023c20     libsetnotif001.obj
 0003:0001ac28       ?endPos@@3PEBEEB           0000000180023c28     libsetnotif001.obj
 0003:0001ac30       ?genPos@@3PEAEEA           0000000180023c30     libsetnotif001.obj
 0003:0001ac38       ?markPos@@3PEAEEA          0000000180023c38     libsetnotif001.obj
 0003:0001ac40       ?constantPool@@3PEAPEADEA  0000000180023c40     libsetnotif001.obj
 0003:0001ac48       ?constantPoolCount@@3GA    0000000180023c48     libsetnotif001.obj
 0003:0001ac4c       ?zeroBytes@@3PAEA          0000000180023c4c     libsetnotif001.obj
 0003:0001ac50       ?codeLength@@3IA           0000000180023c50     libsetnotif001.obj
 0003:0001ac54       result                     0000000180023c54     libsetnotif001.obj
 0003:0001ac58       ?map@@3PEAIEA              0000000180023c58     libsetnotif001.obj
 0003:0001ac60       ?widening@@3PEACEA         0000000180023c60     libsetnotif001.obj
 0003:0001ac68       jvmti                      0000000180023c68     libsetnotif001.obj
 0003:0001ac70       caps                       0000000180023c70     libsetnotif001.obj
 0003:0001ac80       callbacks                  0000000180023c80     libsetnotif001.obj
 0003:0001adb8       access_lock                0000000180023db8     libsetnotif001.obj
 0003:0001adc0       notifyFramePopThread       0000000180023dc0     libsetnotif001.obj
 0003:0001adc8       flag                       0000000180023dc8     libsetnotif001.obj
 0003:0001add0       enbl_scale                 0000000180023dd0     libsetnotif001.obj
 0003:0001ae30       ev_scale                   0000000180023e30     libsetnotif001.obj
 0003:0001aea0       GS_ExceptionRecord         0000000180023ea0     MSVCRT:gs_report.obj
 0003:0001af40       GS_ContextRecord           0000000180023f40     MSVCRT:gs_report.obj
 0003:0001b410       ?g_tss_cv@@3U_RTL_CONDITION_VARIABLE@@A 0000000180024410     MSVCRT:thread_safe_statics.obj
 0003:0001b418       ?g_tss_event@@3PEAXEA      0000000180024418     MSVCRT:thread_safe_statics.obj
 0003:0001b420       ?g_tss_mutex@@3U_RTL_CRITICAL_SECTION@@A 0000000180024420     MSVCRT:thread_safe_statics.obj
 0003:0001b448       ?g_sleep_condition_variable_cs@@3P6AHPEAU_RTL_CONDITION_VARIABLE@@PEAU_RTL_CRITICAL_SECTION@@K@ZEA 0000000180024448     MSVCRT:thread_safe_statics.obj
 0003:0001b450       ?g_wake_all_condition_variable@@3P6AXPEAU_RTL_CONDITION_VARIABLE@@@ZEA 0000000180024450     MSVCRT:thread_safe_statics.obj
 0003:0001b45c       ?__proc_attached@@3HA      000000018002445c     MSVCRT:dll_dllmain.obj
 0003:0001b470       ?is_initialized_as_dll@@3_NA 0000000180024470     MSVCRT:utility.obj
 0003:0001b471       ?module_local_atexit_table_initialized@@3_NA 0000000180024471     MSVCRT:utility.obj
 0003:0001b478       ?module_local_atexit_table@@3U_onexit_table_t@@A 0000000180024478     MSVCRT:utility.obj
 0003:0001b490       ?module_local_at_quick_exit_table@@3U_onexit_table_t@@A 0000000180024490     MSVCRT:utility.obj
